:100000008A0112280C291B292F2944294F296329E9
:100010009129A029F629032A0E2A192A2B2A412AD6
:100020005E2A6D2A02208A110A1207208A110A12FA
:100030003C30FD0006208A110A120F30FD00062018
:100040008A110A12831203138701FA0110208A1100
:100050000A120A208A110A12FB01F50175080F3CE9
:10006000013003190301003C0319A728831203136D
:100070008C1E41281A08F6007608FC0004208A111C
:100080000A1209208A110A12103075020130031871
:100090000301003C03199D28FA080130031D0301E8
:1000A000003C03199C280130FA000A307502013027
:1000B00003180301003C03197228F0017508303E53
:1000C0000318F00AFC0004208A110A12F0017508D6
:1000D000303E0318F00A83120313A00011208A1186
:1000E0000A128628F0017508373E0318F00AFC0052
:1000F00004208A110A12F0017508373E0318F00A2D
:1001000083120313A00011208A110A120B208A11F6
:100110000A12A030FE000D208A110A127B08FE0090
:100120000D208A110A127508FE000D208A110A128C
:100130000C208A110A12FB0AA1287A080319A128A7
:10014000FA010A30F20008208A110A122E28C03063
:10015000FD0006208A110A12FB010A208A110A12E8
:100160000B208A110A12A030FE000D208A110A12FB
:100170007B08FE000D208A110A120C208A110A1237
:100180000B208A110A12A130FE000D208A110A12DA
:10019000F50175080F3C013003190301003C0319F8
:1001A00003290E208A110A12F5000A307502013067
:1001B00003180301003C0319E728F0017508303EDD
:1001C0000318F00AFC0004208A110A12F028F0013A
:1001D0007508373E0318F00AFC0004208A110A1241
:1001E00075080F3C0130031D0301003C0319FE2874
:1001F0000130FF000F208A110A120229FF010F208F
:100200008A110A12C9280C208A110A120230FD0034
:1002100006208A110A122C28831203138501F83054
:100220008316850006309F00831205100511851086
:10023000831686010800FF3083160313860083129D
:100240008514831203130511000005150000861B99
:1002500021290511000085108316860108008312EC
:100260000313851005107C08860003208A110A12EA
:100270008312031305140515000005112D30F40039
:1002800005208A110A120800F40CF40C3F30F40522
:100290000330F4020000F40B4A2900000800831226
:1002A0000313851005107D08860003208A110A12A9
:1002B000831203130515000005112D30F4000520ED
:1002C0008A110A1208003C30FD0006208A110A1229
:1002D0000530F20008208A110A123C30FD00062089
:1002E0008A110A120530F20008208A110A123C30E5
:1002F000FD0006208A110A120530F20008208A113A
:100300000A120830FD0006208A110A120130FD0091
:1003100006208A110A120630FD0006208A110A12F0
:1003200008008E30F3000000000000000000000014
:100330000000F30B95290000F20B91290000080042
:10034000F030831603138600811383128601060999
:10035000F800F80EF70178080139FF390130031D64
:100360000030003C0319B929780C7F39F800F70AEE
:10037000AB2904307702013003180301003C031954
:10038000F3297708F9000F308316031386008113D1
:10039000831286010609F800F70178080139FF3950
:1003A0000130031D0030003C0319DB29780C7F3934
:1003B000F800F70ACD290430770201300318030151
:1003C000003C0319F0297708F800F0017908F100E2
:1003D000F10D710DFC3978070318F00AF500F229C8
:1003E000FF30F500F529FF30F500080083160313F0
:1003F0000708303887008030940009309300283097
:10040000831294000800831203138C1183161114B5
:1004100083160313111C0D2A082A080083120313E4
:100420008C118316111583160313111D182A132A14
:100430000800831203138C117E08930083120313A8
:100440000C080839003C0130031D0301003C03196E
:100450002A2A1E2A0800831203138C118316911571
:10046000831203130C080839003C0130031D0301FB
:10047000003C03193C2A302A831203138C11130801
:100480000800831203138C117F08003C03194B2AC8
:10049000831691164E2A83160313911283160313A3
:1004A0001116831203130C080839003C0130031D98
:1004B0000301003C03195D2A512A080019308316F4
:1004C00003139900A430980090308312980083168B
:1004D0000708BF39803887000800831203132008FB
:0404E0009900080077
:00000001FF
